:10000000B1284108C7004406C8004208031D45083E
:1000100003193628C2077E30031C1228C202031CB3
:1000200015283828C202031C35284008C600C71707
:10003000C417C001C1011030C900C70CC60C031C95
:1000400027284308C00744080318440FC107C10C00
:10005000C00CC90B1D28C11B3E28C00DC10DC20814
:1000600003193528C203470D3E284A15C2013B2813
:10007000CA14FF30C200C0018030C100C81FC113C4
:10008000400808008E30C600C701C21F5028C209B0
:10009000C109C009C00F4F28C10A0319C20AC717F6
:1000A000C20803195A280830C6074108C000420890
:1000B000C1006928C108031D69280830C60240082C
:1000C00003196F28C100C00169280310C00DC10DBC
:1000D000C603C11F65284608C200C71FC1134008D8
:1000E00008004108C6007F304202C700031CA72851
:1000F000C117C20147080F3CC70003188928083000
:10010000C707031CA9284108C2004008C100C0015C
:10011000912808304702031C9128C7004108C000FD
:10012000C101C70803199A280310C20CC10CC00CE6
:10013000C70B9428C21BA928C61FAF28C209C10932
:10014000C009C00FAF28C10A0319C20AAF280001B5
:10015000AB28CA14FF30C200C100C000C21340085F
:1001600008007F230030D0234108CC004208CD0096
:100170004D08031DC2280C304C020318C2280C3055
:10018000CC00CD0103304D02031CD028031DCC2828
:10019000F5304C02031CD028F430CC000330CD00E5
:1001A00002304D020318DE284D08023CAC004C081A
:1001B000003CAB00031CAC035414E42802304D0295
:1001C000AC004C08AB0054102B08C1002C08C20036
:1001D0001030C0000310AB0DAC0DC10DC20D031CDF
:1001E000F5285A30AB070318AC0AC00BEA282B08D5
:1001F000C1002C08C200C3011030C000C10DC20DE7
:10020000C30D0318072932304302031C0A29323078
:10021000C3020314AB0DAC0DC00BFE28541C1929EE
:100220002C08053CAC002B08DC3CAB00031CAC03E9
:100230001F290530AC07DC30AB070318AC0A0130CE
:10024000D0234108CE004208CF004F08031D2F29BC
:100250000C304E0203182F290C30CE00CF01033092
:100260004F02031C3D29031D3929F5304E02031CA2
:100270003D29F430CE000330CF0002304F02031886
:100280004B294F08023CAE004E08003CAD00031C59
:10029000AE035414512902304F02AE004E08AD0097
:1002A00054102D08C1002E08C2001030C0000310E9
:1002B000AD0DAE0DC10DC20D031C62295A30AD0744
:1002C0000318AE0AC00B57292D08C1002E08C20022
:1002D000C3011030C000C10DC20DC30D0318742935
:1002E00032304302031C77293230C3020314AD0DB0
:1002F000AE0DC00B6B29541C86292E08053CAE00A0
:100300002D08DC3CAD00031CAE038C290530AE0784
:10031000DC30AD070318AE0A0230D0234108D0000C
:100320004208D1005108031D9C29103050020318C7
:100330009C291030D000D10103305102031CAA299E
:10034000031DA629F5305002031CAA29F430D00061
:100350000330D10083128519B5290330C000031082
:10036000D10CD00CC00BAF29BB290310D10CD00C81
:100370000310D10CD00C2E082C020319C7292C080D
:100380002E060318803A80390319CB29D5292D0868
:100390002B020318D5292B08A1002C08A2002D0838
:1003A000A3002E08A400D410DE292D08A1002E08D9
:1003B000A2002B08A3002C08A400D4148312101050
:1003C000CF30D2008A30D30053088F0052088E00FD
:1003D0000C1010148312851AEF290C1CEA298312C1
:1003E00010100C18622A83121010CF30D2008A30FD
:1003F000D30053088F0052088E000C101014831283
:10040000851E042A0C1CFF29831210100C18622A66
:1004100083120F08A500A6012508A600A5010E0855
:10042000A504CF30D2008A30D3005308A602520868
:10043000A502031CA603A61BB22803302602031C38
:10044000B228031D272A20302502031CB228A61B30
:10045000332A08302602031C332A031D622A9930EE
:1004600025020318622A03302602031C3D2A031DBD
:10047000412ADC3025020318412ADC30A500033074
:10048000A60007302602031C4F2A031D4B2ADD302D
:100490002502031C4F2ADC30A5000730A60083127A
:1004A0008519702AA61B5E2A05302602031C5E2AC7
:1004B000031D602ADC3025020318602AD411702A3B
:1004C000D415702A8312851D6A2ADC30A5000330FA
:1004D000A600702A8312851A6F2AD411702AD415A7
:1004E00083128519922A54198A2A2308A7002408FE
:1004F000A800822AD415D41C892A2108A700220822
:10050000A800892AD411D418892A2108A700220812
:10051000A8005415D4198F2AD41C372B522BD41869
:10052000372B522B54199A2A2508A7002608A80011
:1005300054156C2B2C082E02B0002B082D02AF0096
:10054000031CB0032F08B1003008B200B301B21B86
:10055000B3033108C0003208C1003308C200422092
:100560004008B7004108B8004208B900033026022D
:10057000B000DC302502AF00031CB0032F08B4002C
:100580003008B500B601B51BB6033408C000350805
:10059000C1003608C20042204008BA004108BB0032
:1005A0004208BC003708C0003808C1003908C20042
:1005B0003A08C3003B08C4003C08C50001204008BD
:1005C000BD004108BE004208BF003D08B7003E081C
:1005D000B8000A303F020318EF2A4A150030B9006C
:1005E0003708C0003808C1003908C200712040082F
:1005F000B1004108B2004208B3003108AF00320830
:10060000B0002C083007AA002B082F07A9000318F8
:10061000AA0A28082A02B00027082902AF00031CF2
:10062000B003B01F182BB009AF09AF0A0319B00A05
:1006300051083002031C222B031D272B50082F02C8
:100640000318272B2908A7002A08A8006C2B2A08C2
:1006500028020319332B2A0828060318803A803908
:100660000319522B372B29082702031C522B510840
:10067000A8025008A702031CA80322082802031995
:10068000492B280822060318803A803903194D2B7C
:100690006C2B2108270203186C2B2108A7002208C5
:1006A000A8006C2B5108A8075008A7070318A80A30
:1006B000280824020319642B280824060318803A0A
:1006C00080390319682B6C2B2708230203186C2B25
:1006D0002308A7002408A800831210102809D300BB
:1006E0002709D20053088F0052088E000C101014F6
:1006F000051683120C1C792B83120512B228FF23D6
:10070000831690003F30CB000130C0000130A92398
:100710000230C0000130A9230430C0000130A923F9
:100720000830C0000030A9231030A2232030C000C0
:100730000030A923C0010130BC2383129001541161
:1007400054120800C0004009CB054B0883168500F1
:100750000800C1004008CB044B0883168500073011
:1007600083129900410BB82B400883169F04BB2BC2
:10077000400983169F050800C10040088312031D2D
:100780001F1703191F134108031D9F1703199F13F8
:100790008F3083169F0550309F0483121F1408006A
:1007A000C00004304002031CD82BC101C201003438
:1007B00083121F119F110310400D400740079F0433
:1007C000000000000000000000009F1483129F182A
:1007D000E62B83121E08C100C2014108C200C101FC
:0C07E00083161E08C10441080800080030
:0E07F000550053004300560030002E0042001A
:02400E0094011B
:00000001FF
